:100000000C942A001895000018950000189500001F
:10001000189500001895000018950000189500002C
:10002000189500000C945F0C1895000018950000BE
:10003000189500001895000018950000189500000C
:1000400018950000189500001895000018950000FC
:10005000189500008FE58DBFC4E0E0E84E2E88E0E3
:100060008EBFD8E0F7E05F2EEEEFF7E0A0E6B0E05D
:1000700088278D933197E9F783E389B980E080BDC4
:1000800088E18AB9662481E48ABB81E38BBB8FEB6C
:1000900087BB8FEB88BB88E084BB83E085BB80E0B7
:1000A00081BB8BE382BB80E08FBD81E08EBD8FE1A1
:1000B00081BD87E181BD86E086B980E487B9C398B8
:1000C000C29AD89ADE9AC498C798C598F894A89509
:1000D0008091CF00877F8093CF008091CF008B7F6E
:1000E0008093CF000027AFECB0E08C9183FB0EF43F
:1000F00001E040E0041711F00C949F0081E48ABBFA
:10010000DC9A82E390E00E94032D379A84E48064B5
:1001100087B90E944B2DA3E6B0E08D939C9337984E
:10012000A3E6B0E00D911C91003052E0150710F0ED
:100130000C949F008091CF0084608093CF000027B3
:10014000AFECB0E08C9183FB0EF401E041E00417CA
:1001500081E009F080E08F930027AFECB0E08C9154
:1001600082FB0EF401E041E0041781E009F080E039
:100170009F91892B882311F40C94C100DC9881E5B0
:100180008ABB0E94CC0D8091CF0080628093CF000B
:10019000EFEFF1E0A0ECB0E091E00E944D2E009175
:1001A000C000003081E009F080E08F930091C00032
:1001B0000E3F80E010F009F081E09F91892B8823A9
:1001C00011F40C94E6008EEB8093C0000091C00007
:1001D0004AE0040F01BF89E190E00E94032DE0EFA7
:1001E000FCE50E94672C0027AFECB0E08C9183FB0C
:1001F0000EF401E041E0041711F00C940701EEE069
:10020000FDE50E94672C0E94732C0C941A01E0E11A
:10021000FDE50E94672CAFECB0E08C9182FBA8E674
:10022000B7E00E94642D8D9388278C930E945F2CE9
:100230000E94732CEAE0F0E0BB27A0E10E944A2E66
:10024000073411F40C945A01EBE0F0E0A0E1BB2775
:100250008FE08C937BE70E94392EECE0F0E001E028
:1002600010E0A0E1BB277BE70E943B2EEAE0F0E034
:10027000A0E1BB2787E48C937BE70E94392EEEE058
:10028000F0E0A0E1BB2780E08C937BE70E94392E51
:10029000E0E1F0E000E010E0A0E1BB277BE70E9496
:1002A0003B2EEFE0F0E0A0E1BB2780E08C937BE702
:1002B0000E94392EEBE0F0E0ABEBB0E00E944A2E5A
:1002C0000091BB00043618F011F00C9469010C94F5
:1002D0006C0184E68093BB0080E797E9ACEBB0E06B
:1002E0008D939C93ECE0F0E0A6EBB0E00E944C2EE6
:1002F000EEE0F0E0A1ECB0E00E944A2EEFE0F0E08A
:10030000A2ECB0E00E944A2E0E94D00DE0E1F0E0A5
:10031000A3E6B0E00E944C2EA3E6B0E00E94DD2BE5
:10032000E0E1F0E0A3E6B0E07BE70E943B2EA6EB25
:10033000B0E00D911C91003050E0150711F00C94C5
:10034000A70181E090E0A6EBB0E08D939C93E2E101
:10035000FDE50E94672CA8E6B7E0EBEBF0E00E9419
:10036000D22D0E945F2CEAE1FDE50E94672CA8E6F1
:10037000B7E0E6EBF0E00E94C32D0E945F2CEAE1BB
:10038000FDE50E94672CA8E6B7E0E1ECF0E00E94F2
:10039000D22D0E945F2CEAE1FDE50E94672CA8E6C1
:1003A000B7E0E2ECF0E00E94D22D0E945F2CEAE17F
:1003B000FDE50E94672CA8E6B7E0E3E6F0E00E94C6
:1003C000C32D0E945F2C0E94732C80E08093CE008E
:1003D00080916A00877F80936A0080E08093C400E8
:1003E00086E08093BE008DE08093BF00E9E6F0E0F8
:1003F000FA93EA930E94121D229684E190E00E94F3
:10040000032DDE980E94EF2CC49AECE1FDE50E94DA
:10041000672C0E94732C88EC90E00E94032DA89515
:1004200081B5886181BD877F81BDE0E6F0E0FA9308
:10043000EA930E945A212296A8950091600000300C
:1004400011F40C942F020E949C20E6E2FDE50E942C
:10045000672C0E94732C0E94930D0C94340280919F
:10046000CF008F7B8093CF00E0E3FDE50E94672CF7
:100470000E94C52084E690E00E94032D009169004F
:10048000003018F011F00C9447020C944E02E9E68B
:10049000F0E0FA93EA930E94A11E22960027AFECA7
:1004A000B0E08C9186FB0EF401E040E0041711F0FF
:1004B0000C945C020E944D148FEF0E94762C82E314
:1004C00090E00E94032D7894A89581B5886081BD45
:1004D000A2EBB0E04D915C91A6EBB0E00D911C91C8
:1004E0000417150718F011F00C9478020C947E0292
:1004F00081E090E0A6EBB0E08D939C930027AAE604
:10050000B0E08C9184FB0EF401E041E0041781E03F
:1005100009F080E08F930027AFECB0E08C9186FB70
:100520000EF401E040E0041781E009F080E09F91C3
:100530008923882311F40C94B002E6EBF0E0FA93DF
:10054000EA935A924A9280E0A42DB52D8C9381E0D3
:100550000E94CA2B0E940D12249681E00E94C62B95
:1005600080E08093B80080E08093690080916A0009
:100570008F7780936A000027AFECB0E08C9186FB08
:100580000EF401E041E0041711F00C94C9020E943E
:10059000CC0DA895ABE6B0E088278C930027AFEC94
:1005A000B0E08C9183FB0EF401E041E0041711F000
:1005B0000C94E1020E94572CABE6B0E08D938827A3
:1005C0008C93ABE6B0E08C91803011F00C94760502
:1005D0000091CE00003081E009F080E08F93002789
:1005E000AAE6B0E08C9181FB0EF401E040E0041734
:1005F00081E009F080E09F91892B882311F40C940D
:100600005A04E0E6F0E0FA93EA930E946A1D22960B
:1006100000916000003018F011F00C9411030C945C
:100620005A0480916A00806880936A000091D0002B
:10063000003011F00C946203809160008093C4003C
:100640000027AAE6B0E08C9184FB0EF401E040E0C4
:10065000041711F00C943C03A0E6B0E08C91A6EBDB
:10066000B0E08D9388278C93ABE6B0E0EAE3FDE53C
:100670000E94452D0C9462030027AFECB0E08C91F2
:1006800087FB0EF401E041E0041711F00C945C03C9
:10069000A0E6B0E00D91112741E050E0040F151FD6
:1006A000A6EBB0E00D931C93ABE6B0E0EAE3FDE50A
:1006B0000E94452D0C946203ABE6B0E0ECE3FDE54F
:1006C0000E94452D0091D000013011F00C94E203FE
:1006D00000916000013011F00C947403ABE6B0E0BF
:1006E000ECE3FDE50E94452D00916000023011F021
:1006F0000C948003ABE6B0E0EEE3FDE50E94452DEF
:1007000080E08093620000916000033081E009F096
:1007100080E08F930091BB00043681E008F080E018
:100720009F918923882311F40C949E03ABEBB0E0D6
:100730008C918E5F8C9381E08093620000916000C9
:10074000043081E009F080E08F930091BB0002301B
:1007500080E010F009F081E09F918923882311F453
:100760000C94BA03ABEBB0E08C9182508C9381E097
:100770008093620000916200013011F00C94E2035A
:100780008EB5887F8EBD5A924A928091BB00A42D6F
:10079000B52D8C9381E00E94CA2B0E944828229696
:1007A00081E00E94C62BEBE0F0E0ABEBB0E07BE732
:1007B0000E94392E0091CE00013011F00C94E2031A
:1007C00081E08EBD0091D000023011F00C945A04EB
:1007D000809160008093C40000916000013011F0AE
:1007E0000C94FE0381E090E0A6EBB0E08D939C9327
:1007F000ABE6B0E0EAE3FDE50E94452D0091600024
:10080000023011F00C944204A2EBB0E00D911C9167
:1008100041E050E0041B150BA3E6B0E00D931C93E0
:1008200002E010E00F931F93A3E6B0E08D919C913E
:100830008A939A930E94F82B2296402F512F1F9152
:100840000F91040F151FA3E6B0E00D931C93A6EBC8
:10085000B0E04D915C91A3E6B0E00D911C910417BE
:10086000150711F40C940404A3E6B0E08D919C915B
:10087000A6EBB0E08D939C93ABE6B0E0EAE3FDE538
:100880000E94452D00916000033011F00C944E043D
:10089000ABE6B0E0ECE3FDE50E94452D0091600081
:1008A000043011F00C945A04ABE6B0E0EEE3FDE541
:1008B0000E94452D0027AAE6B0E08C9184FB0EF43F
:1008C00001E041E0041781E009F080E08F93002708
:1008D000AFECB0E08C9187FB0EF401E041E004172F
:1008E00081E009F080E09F9189238F930091CE00F1
:1008F000013081E009F080E09F918923882311F481
:100900000C94C504A6EBB0E00D911C91013050E0B1
:10091000150711F00C94C504E0E6F0E0FA93EA93B1
:100920000E946A1D229600916000003080E010F065
:1009300009F081E08F93A2EBB0E04D915C91A0E6CD
:10094000B0E00D9111270417150781E008F080E051
:100950009F918923882311F40C94C504A0E6B0E08C
:100960000D91112741E050E0040F151FA6EBB0E0F8
:100970000D931C93ABE6B0E0EAE3FDE50E94452D44
:1009800080916A00806880936A000027AAE6B0E040
:100990008C9180FB0EF401E040E0041711F00C9400
:1009A0007605E9E6F0E0FA93EA930E94121D22969A
:1009B00000916900043011F00C94E5040E94640D6C
:1009C00080916A00806880936A0080E08093600074
:1009D00000916900023081E009F080E08F9300917E
:1009E000BB00043681E008F080E09F9189238823D2
:1009F00011F40C940305ABEBB0E08C918B5F8C93FE
:100A000081E08093600000916900033081E009F08B
:100A100080E08F930091BB00053081E009F080E019
:100A20009F918923882311F40C941C0581E0809305
:100A3000BB0081E08093600000916900033081E099
:100A400009F080E08F930091BB00053080E010F04A
:100A500009F081E09F918923882311F40C943805D3
:100A6000ABEBB0E08C9185508C9381E0809360007B
:100A700000916000013011F00C9465058EB5887FFF
:100A80008EBD5A924A928091BB00A42DB52D8C93B5
:100A900081E00E94CA2B0E944828229681E00E9491
:100AA000C62BEBE0F0E0ABEBB0E07BE70E94392E29
:100AB0000091CE00013011F00C94600581E08EBDF4
:100AC00080916A00806880936A000091690001301B
:100AD00011F00C947605ABE6B0E0ECE3FDE50E9486
:100AE000452D80916A00806880936A00EBE6F0E013
:100AF000ABE6B0E00E94582DABE6B0E08C918030C0
:100B000081E009F480E08F9300916900003081E07A
:100B100009F480E09F91892B8F930091B8000130F8
:100B200081E009F080E09F91892B882311F40C94D7
:100B3000BB020091B800013011F00C94C00580E0B8
:100B40008093B800ABE6B0E0ECE3FDE50E94452DF4
:100B50000027AFECB0E08C9187FB0EF401E041E0A0
:100B6000041711F00C94C00581E090E0A6EBB0E012
:100B70008D939C93ABE6B0E0EAE3FDE50E94452D42
:100B8000ABE6B0E0E0E4FDE50E94642E11F00C94C9
:100B900007065A924A928091BE00A42DB52D8C93DF
:100BA00081E00E94CA2B5A924A928091BF00A42DE4
:100BB000B52D8C9381E00E94CA2B0E94A128249617
:100BC00082E00E94C62B0091C20041E0042BA0E607
:100BD000B0E00C938091CF0080618093CF008EB500
:100BE000887F8EBDEFE0F0E0A0E6B0E07BE70E94FA
:100BF000392E809160008093C2000091CE000130B8
:100C000011F00C94050681E08EBD0C94910BE2E48A
:100C1000FDE50E94642E11F00C944A065A924A9205
:100C200080E0A42DB52D8C9381E00E94CA2B5A92AE
:100C30004A9280E0A42DB52D8C9381E00E94CA2BAE
:100C40000E94A128249682E00E94C62B0091C20037
:100C50004EEF0423A0E6B0E00C938091CF008F7E8E
:100C60008093CF008EB5887F8EBDEFE0F0E0A0E6E8
:100C7000B0E07BE70E94392E809160008093C20033
:100C80000091CE00013011F00C94480681E08EBD39
:100C90000C94910BEAE3FDE50E94642E11F00C9494
:100CA000BA060091CE00013011F00C9459060E9452
:100CB000640DA2EBB0E04D915C91A6EBB0E00D911C
:100CC0001C910417150718F011F00C94B5060027B5
:100CD000AFECB0E08C9186FB0EF401E040E004172D
:100CE00011F00C948606E6EBF0E0FA93EA935A9240
:100CF0004A9280E0A42DB52D8C9381E00E94CA2BEE
:100D00000E940D12249681E00E94C62B0027AFECB2
:100D1000B0E08C9186FB0EF401E041E0041711F085
:100D20000C94B3060E94930D0027AFECB0E08C91B9
:100D300086FB0EF401E040E0041711F00C94B306BA
:100D4000E6EBF0E0FA93EA935A924A9280E0A42DFF
:100D5000B52D8C9381E00E94CA2B0E940D1224961F
:100D600081E00E94C62B0C94B80680E08093C400FA
:100D70000C94910BE4E4FDE50E94642E11F00C94B8
:100D8000C8060E94640D80E08093C4000C94910B0F
:100D9000E6E4FDE50E94642E11F00C940407009136
:100DA000CE00013011F00C9402070027AAE6B0E053
:100DB0008C9183FB0EF401E040E0041711F00C94D9
:100DC000F2068EB5887F8EBD89B78B7F89BF8091F3
:100DD0006A00886080936A0084E690E00E94032D98
:100DE0000C94020780916A00877F80936A0080E2FA
:100DF0009EE490934D0080934C0081E08EBD89B7B6
:100E0000846089BF0C94910BECE3FDE50E94642E95
:100E100011F00C949C070091CE00013011F00C945D
:100E200013070E94640DA6EBB0E00E94DD2B0027A3
:100E3000AFECB0E08C9185FB0EF401E041E00417CB
:100E400011F00C9438070027AAE6B0E08C9184FBDF
:100E50000EF401E040E0041711F00C943307A6EB08
:100E6000B0E00E94E42B8091CF008F7D8093CF0073
:100E7000A2EBB0E04D915C91A6EBB0E00D911C911E
:100E80000417150718F011F00C9448070C944E073E
:100E900081E090E0A6EBB0E08D939C930027AFEC4F
:100EA000B0E08C9186FB0EF401E040E0041711F0F5
:100EB0000C946D07E6EBF0E0FA93EA935A924A92AB
:100EC00080E0A42DB52D8C9381E00E94CA2B0E9456
:100ED0000D12249681E00E94C62B0027AFECB0E0F3
:100EE0008C9186FB0EF401E041E0041711F00C94A4
:100EF0009A070E94930D0027AFECB0E08C9186FB1F
:100F00000EF401E040E0041711F00C949A07E6EBB0
:100F1000F0E0FA93EA935A924A9280E0A42DB52D1C
:100F20008C9381E00E94CA2B0E940D12249681E0CE
:100F30000E94C62B0C94910BEEE3FDE50E94642EFB
:100F400011F00C9414080091CE00013011F00C94B3
:100F5000AB070E94640DA6EBB0E00D911C9101302F
:100F600050E0150718F011F00C94B8070C94BE0768
:100F7000A6EBB0E00E94E42B0C94C607A2EBB0E015
:100F80008D919C91A6EBB0E08D939C930027AFECE4
:100F9000B0E08C9186FB0EF401E040E0041711F004
:100FA0000C94E507E6EBF0E0FA93EA935A924A9242
:100FB00080E0A42DB52D8C9381E00E94CA2B0E9465
:100FC0000D12249681E00E94C62B0027AFECB0E002
:100FD0008C9186FB0EF401E041E0041711F00C94B3
:100FE00012080E94930D0027AFECB0E08C9186FBB5
:100FF0000EF401E040E0041711F00C941208E6EB47
:10100000F0E0FA93EA935A924A9280E0A42DB52D2B
:101010008C9381E00E94CA2B0E940D12249681E0DD
:101020000E94C62B0C94910BE8E4FDE50E94642E0F
:1010300011F00C948708A6EBB0E00E94DD2BA2EB28
:10104000B0E04D915C91A6EBB0E00D911C910417BE
:10105000150718F011F00C942F080C94350881E056
:1010600090E0A6EBB0E08D939C938EB5887F8EBD0B
:10107000A2E7B0E00D911D912D913C91A2E9B0E065
:101080000D931D932D933C930027AFECB0E08C9112
:1010900086FB0EF401E040E0041711F00C947D088B
:1010A0005A924A92A2E9B0E00D911D912D913C9186
:1010B000A42DB52D0D931D932D933C9384E00E9498
:1010C000CA2B5A924A92A6EBB0E08D919C91A42D26
:1010D000B52D8D939C9382E00E94CA2B5A924A921E
:1010E00080E0A42DB52D8C9381E00E94CA2B0E9434
:1010F0005C15269687E00E94C62B0091CE00013039
:1011000011F00C94850881E08EBD0C94910BE0E108
:10111000FDE50E94642E11F00C94FB08A6EBB0E0F4
:101120000D911C91013050E0150718F011F00C944E
:101130009B080C94A108A6EBB0E00E94E42B0C9451
:10114000A908A2EBB0E08D919C91A6EBB0E08D9345
:101150009C938EB5887F8EBDA2E7B0E00D911D9166
:101160002D913C91A2E9B0E00D931D932D933C93FA
:101170000027AFECB0E08C9186FB0EF401E040E07C
:10118000041711F00C94F1085A924A92A2E9B0E0C7
:101190000D911D912D913C91A42DB52D0D931D9375
:1011A0002D933C9384E00E94CA2B5A924A92A6EB5C
:1011B000B0E08D919C91A42DB52D8D939C9382E0F0
:1011C0000E94CA2B5A924A9280E0A42DB52D8C938E
:1011D00081E00E94CA2B0E945C15269687E00E943F
:1011E000C62B0091CE00013011F00C94F90881E07B
:1011F0008EBD0C94910BEAE4FDE50E94642E11F083
:101200000C940B09ECE0F0E0A6EBB0E07BE70E9469
:101210003B2E0C94910BECE4FDE50E94642E11F042
:101220000C941F098DE181BD85E181BD0E94640D93
:1012300081B5886081BD0C941B090C94910BABE6C1
:10124000B0E0EEE4FDE50E94642E81E008F480E069
:101250008F93ABE6B0E0E0E5FDE50E94642E81E00F
:1012600010F009F080E09F918923882311F40C94F9
:10127000F30989B78B7F89BF8EB5887F8EBD0E94A9
:10128000532CA0E6B0E08C9300916000003011F484
:101290000C943F090E94572CA6EBB0E08D93882751
:1012A0008C9380E08093CE0080916A00877F80934A
:1012B0006A00A2EBB0E04D915C91A6EBB0E00D911D
:1012C0001C910417150780E010F009F081E08F935E
:1012D000A6EBB0E00D911C91003050E0150781E0C5
:1012E00009F080E09F91892B882311F40C949309D5
:1012F00081E090E0A6EBB0E08D939C93E6EBF0E00C
:10130000FA93EA935A924A9281E0A42DB52D8C93D8
:1013100081E00E94CA2B0E940D12249681E00E9457
:10132000C62B0C94F1090027AFECB0E08C9186FB42
:101330000EF401E040E0041781E009F080E08F93B3
:10134000ABE6B0E0EEE4FDE50E94642E81E009F03A
:1013500080E09F918923882311F40C94C209E6EB65
:10136000F0E0FA93EA935A924A9281E0A42DB52DC7
:101370008C9381E00E94CA2B0E940D12249681E07A
:101380000E94C62B0027AFECB0E08C9186FB0EF4D8
:1013900001E040E0041781E009F080E08F93ABE6C4
:1013A000B0E0E0E5FDE50E94642E81E009F080E018
:1013B0009F918923882311F40C94F109E6EBF0E066
:1013C000FA93EA935A924A9280E0A42DB52D8C9319
:1013D00081E00E94CA2B0E940D12249681E00E9497
:1013E000C62B0C94910BE2E5FDE50E94642E11F0F2
:1013F0000C942E0A0E94532CA0E6B0E08C9300912E
:101400006000003011F40C94FA090E94572CABEBE9
:10141000B0E08C938EB5887F8EBD5A924A928091AF
:10142000BB00A42DB52D8C9381E00E94CA2B0E9495
:101430004828229681E00E94C62BEBE0F0E0ABEB5F
:10144000B0E07BE70E94392E0091CE00013011F010
:101450000C942C0A81E08EBD0C94910BE4E5FDE523
:101460000E94642E11F00C947C0A0E94532CA0E67A
:10147000B0E08C9300916000003011F40C94350AB8
:101480008091C100809360000E94572CA1ECB0E0D5
:101490008C93A1ECB0E08C918F738C930E94D00D53
:1014A0000091C10040E10423A0E6B0E00C9300915C
:1014B0006000003111F00C94610A0E94CC0D0C9474
:1014C000630A0E94CE0DA1ECB0E08C918F7E8C93CC
:1014D0008EB5887F8EBDEEE0F0E0A1ECB0E07BE75A
:1014E0000E94392E0091CE00013011F00C947A0A3E
:1014F00081E08EBD0C94910BEEE0FDE50E94642E20
:1015000011F00C94E00A0091C1004FE30423A0E61F
:10151000B0E00C930091CE00013011F00C94950ACC
:10152000A0E6B0E08C9180588C930027AFECB0E03F
:101530008C9186FB0EF401E041E0041711F00C944D
:10154000A60AA0E6B0E08C91805C8C930027AAE606
:10155000B0E08C9183FB0EF401E041E0041711F040
:101560000C94B70AA0E6B0E08C91805E8C938091D9
:10157000B600809362008EB5887F8EBD31E0A0E614
:10158000B0E00E946E2C31E0ABEBB0E00E946E2C1C
:1015900031E0A2E6B0E00E946E2C8091B200809310
:1015A000620031E0A2E6B0E00E946E2C0091CE0015
:1015B000013011F00C94DE0A81E08EBD0C94910B89
:1015C000E6E5FDE50E94642E11F00C94630BA5ED99
:1015D000B0E00D911D912D913C91A1EDB0E04D91A8
:1015E0005D916D917C910E94AB2DA5E6B0E00D93CD
:1015F0001D932D933D93A5E6B0E00E94CE2BA5E66A
:10160000B0E00D911D912D913C9140E052E060E0E1
:1016100070E00E94222DA5E6B0E00D931D932D935E
:101620003D93A5E6B0E00D911D912D913C91A3EC69
:10163000B0E04C915527662777270E94832CA5E6BA
:10164000B0E04D935D936D937D93A5E6B0E00D9171
:101650001D912D913C914AE050E060E070E00E94C5
:10166000832CA5E6B0E04D935D936D937D9344E1AB
:1016700050E060E070E0A5E6B0E00D911D912D9185
:101680003C910E94B02D0CF402C00C94510B00E070
:1016900010E020E030E0A5E6B0E00D931D932D931F
:1016A0003C938EB5887F8EBD34E0A5E6B0E00E9405
:1016B0006E2C0091CE00013011F00C94610B81E092
:1016C0008EBD0C94910BE8E5FDE50E94642E11F0AF
:1016D0000C947B0B8EB5887F8EBDA4EAB0E00E948F
:1016E000612C0091CE00013011F00C94790B81E057
:1016F0008EBD0C94910BEAE5FDE50E94642E11F07D
:101700000C94910B8EB5887F8EBD0E94F8140091C9
:10171000CE00013011F00C948F0B81E08EBD0C9443
:10172000910B81E090E00E94032D0027AAE6B0E033
:101730008C9187FB0EF401E040E0041718F011F0E3
:101740000C94A40B0C945D0C00916900003018F00F
:1017500011F00C94AD0B0C94140CA895E0E6F0E09D
:10176000FA93EA930E94121D2296009160000430C1
:1017700011F00C94080C0E94640D80E08093C4006A
:101780000E94CE0D85E090E00E94032D80E08093C2
:101790006200E0E6F0E0FA93EA930E94121D2296BE
:1017A000A2E6B0E08C918F5F8C9388E090E00E947D
:1017B000032D00916000003081E009F080E08F93FC
:1017C00000916200043680E010F009F081E09F9102
:1017D000892B882311F40C94C90B00916200043604
:1017E00018F011F00C94F60B0C94050C81B588617F
:1017F00081BD877F81BDE3E6F0E0FA93EA930E9422
:10180000850E229681B5886081BD80E0809360005E
:1018100081E090E00E94032D00916000003011F003
:101820000C94AD0B0C94530C0091D000013011F0CE
:101830000C944F0C80E090E0A3E6B0E08D939C9375
:10184000E0E6F0E0FA93EA930E946A1D2296A3E68E
:10185000B0E00E94DD2BEF93FF93ECE8F1E00E94F3
:10186000D72CFF91EF9100916000003081E009F0EA
:1018700080E08F93A3E6B0E00D911C91083250E018
:10188000150780E010F009F081E09F91892B8823F3
:1018900011F40C94200C81E090E00E94032D81E073
:1018A00090E00E94032D0091CE00003011F00C94C6
:1018B0005D0C85E090E00E94032D0C94B6020F921F
:1018C0001F922F923F924F925F927F92AF92BF9260
:1018D0000F931F932F933F934F935F936F937F9338
:1018E0008F939F93AF93BF93CF93DF93EF93FF9328
:1018F0008FB78F93F89489B78B7F89BF8EB5887F18
:101900008EBD5A924A9280E092E0A42DB52D8D931F
:101910009C9382E00E94CA2B0E94442B229682E074
:101920000E94C62B0091D9000A3011F00C949A0C39
:101930000E94CC0D0E948E240091D9000A3011F033
:101940000C94A70C0E94CE0D80E08093D900A9EDE5
:10195000B0E08C918F5F8C93A8950027AFECB0E03E
:101960008C9186FB0EF401E040E0041711F00C941A
:10197000CC0C5A924A9280E092E0A42DB52D8D9322
:101980009C9382E00E94CA2B0E94442B229682E004
:101990000E94C62B0E948E24A5EDB0E04D915D9172
:1019A0006D917C91A1EDB0E00D911D912D913C9137
:1019B0000E94B02D80E00CF481E08F930027AFEC03
:1019C000B0E08C9186FB0EF401E040E0041781E06A
:1019D00009F080E09F918923882311F40C94FD0C79
:1019E00080E49CE990934D0080934C0081E08EBD93
:1019F00089B7846089BF0C94460D80E08093CE0047
:101A000080916A00877F80936A000027AFECB0E086
:101A10008C9186FB0EF401E040E0041711F00C9469
:101A20001A0DAAE6B0E08C9184FBA8EBB0E0882701
:101A300080F98C930091C1004FE70423A1E6B0E048
:101A40000C930E94CE0D80E08093C4000027AFEC81
:101A5000B0E08C9183FB0EF401E041E0041781E0DB
:101A600009F080E08F930027AFECB0E08C9182FB0F
:101A70000EF401E041E0041781E009F080E09F915D
:101A8000892B882311F40C94460DDC988F918FBF1D
:101A9000FF91EF91DF91CF91BF91AF919F918F9186
:101AA0007F916F915F914F913F912F911F910F9176
:101AB000BF90AF907F905F904F903F902F901F907E
:101AC0000F901895F894FFCF89B78B7F89BF8EB59B
:101AD000887F8EBD80E08093CE0080916A00877FF2
:101AE00080936A000027AFECB0E08C9183FB0EF48A
:101AF00001E041E0041781E009F080E08F930027C6
:101B0000AFECB0E08C9182FB0EF401E041E00417F1
:101B100081E009F080E09F91892B882311F40C94D7
:101B2000920DDC980895DE9A6E98C498C598C7986F
:101B30000E94CE0DE2E0F0E00E947A2CDE98C49A7A
:101B40000E94EF2C84E690E00E94032DA8958091DE
:101B5000CF008F7B8093CF00E0E6F0E0FA93EA932A
:101B60000E945A21229600916000003011F40C94DA
:101B7000C90D8091CF0080648093CF0084E690E00F
:101B80000E94032DDE9A6E98C498C598C7980C944D
:101B9000CB0D0E944D140895AB980895AB9A08950B
:101BA00081E00E94122D80916A008F7E80936A00EE
:101BB0000091C10041E00423A881B9810C93A88160
:101BC000B9810C91003011F40C94EB0D80916A00F6
:101BD000806180936A008091CF008F778093CF00DF
:101BE0000091C10042E00423A881B9810C93A8812F
:101BF000B9810C91003011F40C94030E8091CF0048
:101C000080688093CF0080916A008E7F80936A0005
:101C10000091C10044E00423A881B9810C93A881FC
:101C2000B9810C91003011F40C941B0E80916A0064
:101C3000816080936A0080916A008D7F80936A0042
:101C40000091C10048E00423A881B9810C93A881C8
:101C5000B9810C91003011F40C94330E80916A001C
:101C6000826080936A0080916A008F7D80936A0011
:101C70000091C10040E20423A881B9810C93A8819E
:101C8000B9810C91003011F40C944B0E80916A00D4
:101C9000806280936A008091CF008F7E8093CF0016
:101CA0000091C20041E00423A881B9810C93A8816E
:101CB000B9810C91003011F40C94630E8091CF0027
:101CC00080618093CF000091C20046E00423A88188
:101CD000B9810C93A881B9810C9142E00E94542EE5
:101CE0000C93A881B9818C918093D0000091D00091
:101CF000033011F00C947F0E82E08093D00081E0DD
:101D0000481A8827580A2296089582E00E94122DC8
:101D100081E00E94122D81E00E94122D80E0AA81B4
:101D2000BB818C9383E4ACE9B0E08C938FE4ADE9A4
:101D3000B0E08C938EE4AEE9B0E08C9386E4AFE93A
:101D4000B0E08C9389E4A0EAB0E08C93AAE6B0E01E
:101D50008C9185FBA881B981882780F98C9380912B
:101D60006A00806280936A00A2E7B0E00D911D9145
:101D70002D913C91A2E9B0E00D931D932D933C93DE
:101D80005A924A92A2E9B0E00D911D912D913C9199
:101D9000A42DB52D0D931D932D933C9384E00E94AB
:101DA000CA2B5A924A9280E090E0A42DB52D8D93D3
:101DB0009C9382E00E94CA2B5A924A9281E0A42D01
:101DC000B52D8C9381E00E94CA2B0E945C1526964B
:101DD00087E00E94C62B8FE00E94122DE4EAF0E01B
:101DE00006E0A881B9810E942B2EA881B981ECE57B
:101DF000FDE50E94642E0FB68FE0481A8827580A26
:101E000022960FBE81E009F080E08F9300918D0053
:101E1000003181E009F080E09F918923882311F44B
:101E20000C94600F81E0AA81BB818C93A2E9B0E0A1
:101E30000D911D912D913C91A2E7B0E00D931D9362
:101E40002D933C9380916A008F7D80936A005A9213
:101E50004A92A2E9B0E00D911D912D913C91A42DE3
:101E6000B52D0D931D932D933C9384E00E94CA2BB6
:101E70005A924A9280E090E0A42DB52D8D939C93C8
:101E800082E00E94CA2B5A924A9280E0A42DB52D7E
:101E90008C9381E00E94CA2B0E945C15269687E0F5
:101EA0000E94C62BA2E9B0E00D911D912D913C91AD
:101EB000A2E7B0E00D931D932D933C930E94BA0FBF
:101EC000A881B9818C9180FBAAE6B0E08C9185F95C
:101ED0008C93A6E7B0E00D911D912D913C91A2E766
:101EE000B0E00D931D932D933C93A2E7B0E00D91CC
:101EF0001D912D913C91A2E9B0E00D931D932D937E
:101F00003C935A924A92A2E9B0E00D911D912D9115
:101F10003C91A42DB52D0D931D932D933C9384E0FE
:101F20000E94CA2B5A924A9280E090E0A42DB52DCF
:101F30008D939C9382E00E94CA2B5A924A9280E031
:101F4000A42DB52D8C9381E00E94CA2B0E945C15B4
:101F5000269687E00E94C62BAA81BB818C91AE8118
:101F6000BF818D9388278C9384E0481A8827580A6C
:101F70002696089582E00E94122D81E00E94122D83
:101F800081E00E94122D789481E090E0AC81BD81C7
:101F90008D939C93EA81FB81FA93EA93EE81FF8112
:101FA000FA93EA930E94D0112496AA81BB810C91E6
:101FB000013011F00C94E70F82E090E0AC81BD811C
:101FC0008D939C9381E08093C1000C9403100230A8
:101FD00011F00C94F60F83E090E0AC81BD818D93FD
:101FE0009C9380E08093C1000C940310033011F0A7
:101FF0000C94031084E090E0AC81BD818D939C93A0
:1020000083E08093C100EEE0F0E0A1ECB0E07BE77C
:102010000E94392EEC81FD81FA93EA935A924A92FA
:1020200080E0A42DB52D8C9381E00E94CA2B0E94E4
:102030000D12249681E00E94C62B0091CE00003044
:1020400011F00C941D1088EC90E00E94032D85E0A7
:1020500090E0AC81BD818D939C93EA81FB81FA93E2
:10206000EA93EE81FF81FA93EA930E94D0112496BD
:10207000EEE0F0E0A1ECB0E00E944A2EAA81BB8124
:102080000C91033011F00C9447100C94E410AA81C9
:10209000BB810C91013011F00C945510A1ECB0E013
:1020A0008C9188608C930C945E10023011F00C942B
:1020B0005E10A1ECB0E08C91877F8C93EEE0F0E0B5
:1020C000A1ECB0E07BE70E94392E88EC90E00E9402
:1020D000032D86E090E0AC81BD818D939C93EA81D5
:1020E000FB81FA93EA93EE81FF81FA93EA930E94CF
:1020F000D0112496AA81BB810C91033011F00C946D
:1021000083100C94E410EEE0F0E0A1ECB0E00E944B
:102110004A2EAA81BB810C91013011F00C949710CA
:10212000A1ECB0E08C9184608C930C94A0100230F0
:1021300011F00C94A010A1ECB0E08C918B7F8C93EB
:10214000EEE0F0E0A1ECB0E07BE70E94392E88ECF5
:1021500090E00E94032D87E090E0AC81BD818D93DB
:102160009C93EA81FB81FA93EA93EE81FF81FA93D3
:10217000EA930E94D0112496EEE0F0E0A1ECB0E0EA
:102180000E944A2EAA81BB810C91013011F00C945F
:10219000D010A1ECB0E08C9180628C930C94D9109B
:1021A000023011F00C94D910A1ECB0E08C918F7D2D
:1021B0008C93EEE0F0E0A1ECB0E07BE70E94392EDA
:1021C00088EC90E00E94032D88E090E0AC81BD8116
:1021D0008D939C93EC81FD81FA93EA930E94AE115A
:1021E00022960091C10043E00423A881B9810C9399
:1021F000A881B9810C91003011F00C94071183E093
:1022000090E0AC81BD818D939C930C941D110130A5
:1022100011F00C94131182E090E0AC81BD818D939C
:102220009C930C941D11033011F00C941D1184E04B
:1022300090E0AC81BD818D939C93EC81FD81FA93FC
:10224000EA930E94AE1122960091C10048E0042357
:10225000A881B9810C93A881B9810C91003011F04B
:102260000C943A118AE090E0AC81BD818D939C93EF
:102270000C944411083011F00C94441189E090E062
:10228000AC81BD818D939C93EC81FD81FA93EA939F
:102290000E94AE1122960091C10044E00423A8815F
:1022A000B9810C93A881B9810C91003011F00C9484
:1022B00061118BE090E0AC81BD818D939C930C9477
:1022C0006B11043011F00C946B118CE090E0AC8138
:1022D000BD818D939C93EC81FD81FA93EA930E94DA
:1022E000AE1122960091C10040E20423A881B98179
:1022F0000C93A881B9810C91003011F00C948811D5
:102300008DE090E0AC81BD818D939C930C949211F3
:10231000003211F00C9492118EE090E0AC81BD81FE
:102320008D939C93EC81FD81FA93EA930E94AE1108
:1023300022968FE090E0AC81BD818D939C93EC81DF
:10234000FD81FA93EA930E94AE1122960E94D00D6D
:1023500084E0481A8827580A26960895E881F9816A
:10236000FA93EA935A924A9280E0A42DB52D8C9369
:1023700081E00E94CA2B0E940D12249681E00E94E7
:10238000C62B82E390E00E94032D0091CE00003026
:1023900011F00C94C51182E390E00E94032D089582
:1023A00081E00E94122DEA81FB81FA93EA935A920E
:1023B0004A9280E0A42DB52D8C9381E00E94CA2B17
:1023C0000E940D12249681E00E94C62B84E690E0C4
:1023D0000E94032DE881F981FA93EA930E94121D6D
:1023E0002296A881B9810C91003018F011F00C945C
:1023F000FB110C94EA110E94640D84E190E00E94AC
:10240000032DA881B9818C91AC81BD818C9381E031
:10241000481A8827580A2296089582E00E94122DB1
:1024200081E00E94122D8EB5887F8EBD80916A005A
:10243000877F80936A00A2E7B0E00D911D912D91F6
:102440003C91A2E9B0E00D931D932D933C935A92D9
:102450004A92A2E9B0E00D911D912D913C91A42DDD
:10246000B52D0D931D932D933C9384E00E94CA2BB0
:102470005A924A92AA85BB858D919C91A42DB52D27
:102480008D939C9382E00E94CA2B5A924A9280E0DC
:10249000A42DB52D8C9381E00E94CA2B0E945C155F
:1024A000269687E00E94C62B40E050E060E070E096
:1024B000AEE8B0E00D911D912D913C910E94B02DA0
:1024C00011F00C9465120C9447140E94FC275A9248
:1024D0004A928091BB00A42DB52D8C9381E00E947F
:1024E000CA2B0E944828229681E00E94C62B5A924D
:1024F0004A92ACEBB0E08D919C91A42DB52D8D93BB
:102500009C9382E00E94CA2B0E94E028229682E0DF
:102510000E94C62B0027AFECB0E08C9184FB0EF438
:1025200001E041E0041711F00C94B0125A924A9263
:102530008091BE00A42DB52D8C9381E00E94CA2B02
:102540005A924A928091BF00A42DB52D8C9381E0C0
:102550000E94CA2B0E94A128249682E00E94C62BCA
:10256000A2E9B0E00D911D912D913C91A1EDB0E05B
:102570000D931D932D933C93A2E9B0E00D911D9115
:102580002D913C91AEE8B0E04D915D916D917C91C3
:102590000E94A62DA5EDB0E00D931D932D933D93C4
:1025A00080E0A881B9818C930E948E2481E090E024
:1025B000AA81BB818D939C93AA81BB810D911C91B3
:1025C0000F3F51E0150718F011F00C941613AA8173
:1025D000BB81AD90BC90A9EDB0E0AA0DBB1D0C91E4
:1025E0000F3F81E009F080E08F93AA81BB81AD901D
:1025F000BC90AAEDB0E0AA0DBB1D0C910F3E80E08F
:1026000010F009F081E09F918923882311F40C9444
:102610000F1381E0A881B9818C930C941613AA81C1
:10262000BB810E94DD2B10F40C94DC12A881B981CF
:102630000C91013011F00C94D412AA81BB81AD90A1
:10264000BC90ABEDB0E0AA0DBB1D8C91AA81BB8103
:102650008D9388278C93AA81BB810D911C9140E1B9
:1026600050E00E94322CAA81BB814D935C9380E1A3
:102670008093C300AA81BB810D911C91013050E071
:10268000150711F00C94491384E08093C3000C9457
:10269000D613023050E0150711F00C94541385E066
:1026A0008093C3000C94D613033050E0150711F04B
:1026B0000C945F1386E08093C3000C94D61304300F
:1026C00050E0150711F00C946A1387E08093C30063
:1026D0000C94D613053050E0150711F00C947513C7
:1026E00088E08093C3000C94D613063050E01507A1
:1026F00011F00C9480138AE08093C3000C94D613DD
:10270000073050E0150711F00C948B138CE0809388
:10271000C3000C94D613083050E0150711F00C9448
:1027200096138EE08093C3000C94D613093050E0CA
:10273000150711F00C94A11380E18093C3000C9451
:10274000D6130A3050E0150711F00C94AC1384E155
:102750008093C3000C94D6130B3050E0150711F092
:102760000C94B71388E18093C3000C94D6130C30FB
:1027700050E0150711F00C94C2138CE18093C30054
:102780000C94D6130D3050E0150711F00C94CD13B6
:1027900080E28093C3000C94D6130E3050E01507EE
:1027A00011F00C94D61388E28093C300AEE8B0E039
:1027B0000D911D912D913C9140E052E060E070E060
:1027C0000E94222DA5E6B0E00D931D932D933D931D
:1027D000A5E6B0E00D911D912D913C91A3ECB0E0E8
:1027E0004C915527662777270E94832CA5E6B0E0F9
:1027F0004D935D936D937D93A5E6B0E00D911D9192
:102800002D913C9148EE53E060E070E00E94832CF3
:10281000A5E6B0E04D935D936D937D93AC81BD8152
:102820000C91003011F00C94471481E08093CE009D
:1028300088EC9FEA90934D0080934C0089B78460A8
:1028400089BF81E08EBD0027AFECB0E08C9183FBA7
:102850000EF401E041E0041781E009F080E08F937D
:102860000027AFECB0E08C9182FB0EF401E041E078
:10287000041781E009F080E09F91892B882311F4EF
:102880000C944314DC9A85E090E00E94032D83E0D1
:10289000481A8827580A24960895A895A2E7B0E018
:1028A0000D911D912D913C91A6E7B0E00D931D93E4
:1028B0002D933C93A2E7B0E00D911D912D913C9199
:1028C000A2E9B0E00D931D932D933C935A924A9246
:1028D000A2E9B0E00D911D912D913C91A42DB52D53
:1028E0000D931D932D933C9384E00E94CA2B5A9222
:1028F0004A9280E090E0A42DB52D8D939C9382E0C8
:102900000E94CA2B5A924A9280E0A42DB52D8C9336
:1029100081E00E94CA2B0E945C15269687E00E94E7
:10292000C62BA895A2EBB0E00D911C91013050E0B0
:10293000150710F00C94C3145A924A9281E0A42D0A
:10294000B52D8C9381E00E94CA2B0E943A292296D1
:1029500081E00E94C62B8CE291E00E94032D5A92E6
:102960004A9280E0A42DB52D8C9381E00E94CA2B61
:102970000E943A29229681E00E94C62B8091CF00C6
:1029800080648093CF00A895A2E7B0E00D911D91DF
:102990002D913C91A2E9B0E00D931D932D933C93B2
:1029A000A6EBB0E00D911C91003050E0150781E0DE
:1029B00009F080E08F93A2EBB0E04D915C91A6EB23
:1029C000B0E00D911C910417150780E010F009F09C
:1029D00081E09F91892B882311F40C94F51481E0F8
:1029E00090E0A6EBB0E08D939C930E94CE0D0895ED
:1029F00084E00E94122DA1EDB0E00D911D912D916A
:102A00003C91A881B9810D931D932D933C93A2E72E
:102A1000B0E00D911D912D913C91A2E9B0E00D9394
:102A20001D932D933C935A924A92A2E9B0E00D91E6
:102A30001D912D913C91A42DB52D0D931D932D939A
:102A40003C9384E00E94CA2B5A924A928FE19EE402
:102A5000A42DB52D8D939C9382E00E94CA2B5A928F
:102A60004A9280E0A42DB52D8C9381E00E94CA2B60
:102A70000E945C15269687E00E94C62BA2E7B0E074
:102A80000D911D912D913C91A2E9B0E00D931D9304
:102A90002D933C93A881B9810D911D912D913C916D
:102AA000A1EDB0E00D931D932D933C9384E0481A63
:102AB0008827580A2296089581E00E94122D81E00D
:102AC0000E94122D81E00E94122D80E090E0A4EB84
:102AD000B0E08D939C9380916A008F7B80936A0015
:102AE00000E010E020E030E0AEE8B0E00D931D9390
:102AF0002D933C930027AAE6B0E08C9185FB0EF461
:102B000001E041E0041781E009F080E08F93A8859F
:102B1000B9850D911C91003050E0150781E009F452
:102B200080E09F9189238F93AE81BF810C9100300B
:102B300081E009F080E09F918923882311F40C94AF
:102B4000FC15A6E9B0E0E885F9850E94C32DE6E909
:102B5000F0E0A8E6B7E00E941F2EE8E6F7E0A6E95D
:102B6000B0E01127222704E033270E94682D81E47A
:102B7000AC81BD818C93AC81BD818C9180939C0094
:102B800081E0E6E9F0E001E00A93ABE6B0E00E9404
:102B9000242EABE6B0E08C91ADE9B0E08C9382E0FE
:102BA000E6E9F0E001E00A93ABE6B0E00E94242EF3
:102BB000ABE6B0E08C91AEE9B0E08C9383E0E6E95F
:102BC000F0E001E00A93ABE6B0E00E94242EABE611
:102BD000B0E08C91AFE9B0E08C9384E0E6E9F0E0FE
:102BE00001E00A93ABE6B0E00E94242EABE6B0E031
:102BF0008C91A0EAB0E08C9389B78B7F89BF8EB5AA
:102C0000887F8EBD81B5886181BD877F81BDAAEC3B
:102C1000B0E00D911D912D913C91A6ECB0E00D938B
:102C20001D932D933C93A6E7B0E04D915D916D917E
:102C30007C91A2E7B0E00D911D912D913C910E94F5
:102C4000B02D11F00C942E1602E010E020E030E0E0
:102C5000A6ECB0E00D931D932D933C9380E0A881EA
:102C6000B9818C93EA81FB81FA93EA935A924A9252
:102C7000AE85BF850D911D912D913C91A42DB52D53
:102C80000D931D932D933C9384E00E94CA2B0E94C8
:102C90008526249684E00E94C62BAA81BB810C91D4
:102CA0000E3F11F40C9460168091CF0080648093E5
:102CB000CF0080916A00806480936A000C94731640
:102CC0005A924A92AA85BB858D919C91A42DB52DCF
:102CD0008D939C9382E00E94CA2B0E9476172296C5
:102CE00082E00E94C62BA881B9818C918F5F8C9362
:102CF00040916F00A881B9810C91041781E009F01F
:102D000080E08F930027AAE6B0E08C9186FB0EF45A
:102D100001E041E0041781E009F480E09F918923FC
:102D2000882311F40C94291700917E000B3011F0C8
:102D30000C94D616E6ECF0E0FA93EA935A924A9293
:102D4000A6ECB0E00D911D912D913C91A42DB52DD7
:102D50000D931D932D933C9384E00E94CA2B0E94F7
:102D6000B61B249684E00E94C62BEA85FB85FA9365
:102D7000EA935A924A92A6ECB0E00D911D912D91E2
:102D80003C91A42DB52D0D931D932D933C9384E080
:102D90000E94CA2B0E944C1B249684E00E94C62BE2
:102DA00080E0A881B9818C930C942717A6E7B0E046
:102DB0004D915D916D917C91A2E7B0E00D911D91D7
:102DC0002D913C910E94B02D11F00C94ED16AA8526
:102DD000BB850E94CE2B0C942717E6ECF0E0FA930B
:102DE000EA935A924A92A6ECB0E00D911D912D9172
:102DF0003C91A42DB52D0D931D932D933C9384E010
:102E00000E94CA2B0E94B61B249684E00E94C62B07
:102E1000EA85FB85FA93EA935A924A92A6ECB0E0CF
:102E20000D911D912D913C91A42DB52D0D931D93C8
:102E30002D933C9384E00E94CA2B0E944C1B249645
:102E400084E00E94C62B80E0A881B9818C930C9409
:102E50002D17AA85BB850E94CE2B0027AAE6B0E0DD
:102E60008C9186FB0EF401E041E0041711F00C9404
:102E70003216C49AA885B9850D911C91003050E096
:102E8000150711F00C944C17A4EBB0E08D919C91B8
:102E9000A2EBB0E08D939C930091CE00013081E0D5
:102EA00009F080E08F930027AFECB0E08C9186FBB7
:102EB0000EF401E040E0041781E009F080E09F910A
:102EC0008923882311F40C94701780E593EC909378
:102ED0004D0080934C0081E08EBD89B7846089BF2E
:102EE00083E0481A8827580A2696089584E00E94AD
:102EF000122D84E00E94122D81E00E94122D81E0AB
:102F00000E94122D81E00E94122D81E00E94122D5C
:102F100080E0AE81BF818C93AE81BF810C910F3078
:102F200018F011F00C94591981E0AC81BD818C939B
:102F3000AC81BD810C910C3018F011F00C94B817D5
:102F40008FEF0E94F62C0E94F82C0E94F72CAC8187
:102F5000BD81AD90BB24A0E8B0E0AA0DBB1D8C9351
:102F6000AC81BD818C918F5F8C9310F40C94981779
:102F70008DE0AC81BD818C93AC81BD810C9104311D
:102F800018F011F00C94D6178FEF0E94F62C0E94C7
:102F9000F82C0E94F72CA881B9818C93AC81BD815B
:102FA0008C918F5F8C9310F40C94BC17EA85FB8591
:102FB000FA93EA93EA85FB85FA93EA930E94E11972
:102FC00024960027AAE6B0E08C9186FB0EF401E07F
:102FD00041E0041711F00C94EF170C94511980E0A4
:102FE000AA81BB818C9300918C00003281E009F0B2
:102FF00080E08F9300918C00003181E009F080E047
:103000009F91892B882311F40C940A1881E0AA81DE
:10301000BB818C9300918100003081E009F480E055
:103020008F9300918100053E81E009F480E09F913B
:1030300089238F93AA81BB810C91013081E009F033
:1030400080E09F918923882311F40C944619009104
:103050008C00003211F00C943118A4EBB0E00E9407
:10306000DD2B0027AAE6B0E08C9185FB0EF401E091
:1030700040E0041711F00C94661881E0AC81BD812A
:103080008C93AC85BD854D915C91A4EBB0E00D9126
:103090001C910417150781E009F080E08F93A4EBE1
:1030A000B0E00D911C91003050E0150780E010F069
:1030B00009F081E09F918923882311F40C9464180E
:1030C00080E0AC81BD818C930C949A1880E0AC8137
:1030D000BD818C9381E0A881B9818C93A881B9814D
:1030E0000C91053018F011F00C949A18A881B98150
:1030F000AD90BB24ABE9B0E0AA0DBB1D4C91A881FB
:10310000B981AD90BB24A0E8B0E0AA0DBB1D0C9125
:10311000041711F40C94921881E0AC81BD818C935A
:103120000C949A18A881B9818C918F5F8C9310F4BC
:103130000C946E18AC81BD810C91003081E009F0D7
:1031400080E08F93AC85BD850D911C910F315EE4BD
:10315000150781E009F080E09F91892B882311F405
:103160000C9446190E947319A885B9850D911D917B
:103170002D913C9140E052E060E070E00E94832C91
:10318000AEE8B0E04D935D936D937D93E2E9F0E09E
:10319000FA93EA935A924A92AE85BF850D911D919A
:1031A0002D913C91A42DB52D0D931D932D933C9302
:1031B00084E00E94CA2B0E944C1B249684E00E944B
:1031C000C62B80918C0080938D00AC85BD850D91C0
:1031D0001C910F315EE4150711F00C941719A8E645
:1031E000B7E0E4EBF0E00E94C32D0E945F2CE4E620
:1031F000FDE50E94672CA4EAB0E00E94612CE4E6A1
:10320000FDE50E94672C00918C00003111F00C94B8
:103210000D19E6E6FDE50E94672CA8E6B7E0E88513
:10322000F9850E94C62D0E945F2C0E94732CAC81F0
:10323000BD810C91003011F00C94461980916A0008
:10324000806480936A0000918D00003181E009F074
:1032500080E08F93AC85BD850D911C910F315EE4AC
:10326000150781E009F480E09F918923882311F4F8
:103270000C944619AA85BB850D911D912D913C9109
:10328000AAECB0E00D931D932D933C930091810027
:10329000003011F00C94511980916A008064809381
:1032A0006A00AE81BF818C918F5F8C9310F40C9477
:1032B0008C178FEF0E94F62C0E94F82C0E94F72C9E
:1032C000A0E6B0E08C938FEF0E94F62C0E94F82CC1
:1032D0000E94F72CA0E6B0E08C938CE0481A882777
:1032E000580A2C96089581E00E94122DA4EAB0E0BD
:1032F00088278C9381E0A881B9818C93A881B981BA
:103300000C91083018F011F00C94AD19A881B98116
:10331000AD90BB24A0E8B0E0AA0DBB1D0C9100321B
:1033200011F40C94A519A881B981AD90BB24A0E833
:10333000B0E0AA0DBB1D8C91A4EAB0E08F930E946F
:103340004C2C8F918D9388278C93A881B9818C9177
:103350008F5F8C9310F40C947E19A4EAB0E00E9465
:103360004C2CEAE6FDE50E94452D89E0A881B98153
:103370008C93A881B9810C910B3018F011F00C944A
:10338000DB19A881B981AD90BB24A0E8B0E0AA0DFB
:10339000BB1D8C91A4EAB0E08F930E944C2C8F91BE
:1033A0008D9388278C93A881B9818C918F5F8C93A2
:1033B00010F40C94B91981E0481A8827580A22960B
:1033C000089581E00E94122D81E00E94122D84E078
:1033D0000E94122D8FEF0E94F62C0E94F82C0E9462
:1033E000F72CAC81BD818C938FEF0E94F62C0E944C
:1033F000F82C0E94F72CAA81BB818C93AA81BB81F7
:103400000C9111272227332740E051E060E070E063
:103410000E94222DA885B9850D931D932D933D9370
:10342000A885B9850D911D912D913C91AC81BD81EF
:103430004C915527662777270E94A62DA885B98528
:103440000D931D932D933D93A885B9850D911D91E5
:103450002D913C9140E050E061E070E00E94222D0F
:10346000A881B9810D931D932D933D938FEF0E94F9
:10347000F62C0E94F82C0E94F72CAC81BD818C9315
:103480008FEF0E94F62C0E94F82C0E94F72CAC8142
:10349000BD818C938FEF0E94F62C0E94F82C0E9425
:1034A000F72CAC81BD818C938FEF0E94F62C0E948B
:1034B000F82C0E94F72CAC81BD818C938FEF0E9479
:1034C000F62C0E94F82C0E94F72CAC81BD818C93C5
:1034D0008FEF0E94F62C0E94F82C0E94F72CAA81F4
:1034E000BB818C93AA81BB810C91112722273327A2
:1034F00040E051E060E070E00E94222DA885B9858F
:103500000D931D932D933D93A885B9850D911D9124
:103510002D913C91AC81BD814C9155276627772731
:103520000E94A62DA885B9850D931D932D933D93DB
:10353000A885B9850D911D912D913C91A881B981E6
:103540004D915D916D917C910E94A62DA885B985C4
:103550000D931D932D933D938FEF0E94F62C0E94A7
:10356000F82C0E94F72CAC81BD818C938FEF0E94C8
:10357000F62C0E94F82C0E94F72CAA81BB818C9318
:10358000AA81BB810C9111272227332740E051E00B
:1035900060E070E00E94222DA881B9810D931D93F7
:1035A0002D933D93A881B9810D911D912D913C9151
:1035B000AC81BD814C915527662777270E94A62DA7
:1035C000A881B9810D931D932D933D938FEF0E9498
:1035D000F62C0E94F82C0E94F72CAC81BD818C93B4
:1035E0008FEF0E94F62C0E94F82C0E94F72CAA81E3
:1035F000BB818C93AA81BB810C9111272227332791
:1036000040E051E060E070E00E94222DAE81BF8179
:103610000D931D932D933D93AE81BF810D911D910F
:103620002D913C91AC81BD814C9155276627772720
:103630000E94A62DAE81BF810D931D932D933D93C6
:10364000AE81BF810D911D912D913C9140E050E0E4
:1036500061E070E00E94222DAE81BF810D931D9329
:103660002D933D93AE81BF810D911D912D913C9184
:10367000A881B9814D915D916D917C910E94A62D9B
:10368000AE81BF810D931D932D933D9386E0481A23
:103690008827580A2696089584E00E94122D84E017
:1036A0000E94122DAC81BD810D911D912D913C91F7
:1036B00042E050E060E070E00E94AB2DA881B9814B
:1036C0000D931D932D933D93AFE6B0E00C91112720
:1036D00022273327A881B9814D915D916D917C910D
:1036E0000E94222DAA81BB810D931D932D933D93A2
:1036F000AA81BB810D911D912D913C91A6E7B0E06F
:103700004D915D916D917C910E94A62DAA81BB8106
:103710000D931D932D933D9300917E000B3011F47A
:103720000C94A41BAA81BB810D911D912D913C91FC
:1037300040E250E060E070E00E94A62DAA81BB81CB
:103740000D931D932D933D93AA81BB810D911D91E6
:103750002D913C91AE81BF810D931D932D933C9390
:1037600088E0481A8827580A2496089584E00E9421
:10377000122D82E00E94122D00917E000B3011F07C
:103780000C94FA1BAC81BD810D911D912D913C9142
:1037900040E850E060E070E00E94832CA1EDB0E0D2
:1037A0004D935D936D937D93AC81BD810D911C9183
:1037B00040E850E00E94322CA881B9810D931C93FF
:1037C000A881B9810D911C9144E050E00E94182D10
:1037D000A881B9810D931C93A881B9810D911C9189
:1037E00044E050E0040F151FA881B9810D931C938C
:1037F0000C94301CAC81BD810D911D912D913C919B
:1038000040E051E060E070E00E94832CA1EDB0E068
:103810004D935D936D937D93AC81BD810D911C9112
:1038200040E051E00E94322CA881B9810D931C9395
:10383000A881B9810D911C9142E050E00E94182DA1
:10384000A881B9810D931C93A881B9810D911C9118
:1038500042E050E0040F151FA881B9810D931C931D
:10386000A1EDB0E00D911D912D913C91AAE7B0E042
:103870004D915D916D917C910E94A62DA1EDB0E0DE
:103880000D931D932D933D93A1EDB0E00D911D91EE
:103890002D913C91ADE6B0E04D915C916627772784
:1038A0000E94A62DA1EDB0E00D931D932D933D93A5
:1038B0000E948E24A881B981AD90BC90A9EDB0E0A2
:1038C000AA0DBB1D8C91AA81BB818D9388278D93F6
:1038D0008D938C93A881B9810E94E42BAA81BB812E
:1038E0000D911D912D913C9140E051E060E070E020
:1038F0000E94222DAA81BB810D931D932D933D9390
:10390000AA81BB810D911D912D913C91A881B98116
:10391000AD90BC90A9EDB0E0AA0DBB1D4C91552710
:10392000662777270E94A62DAA81BB810D931D9340
:103930002D933D9300917E000B3011F00C94001DEF
:10394000A881B9810E94E42BAA81BB810D911D91B0
:103950002D913C9140E051E060E070E00E94222D0A
:10396000AA81BB810D931D932D933D93AA81BB81A9
:103970000D911D912D913C91A881B981AD90BC9084
:10398000A9EDB0E0AA0DBB1D4C91552766277727FE
:103990000E94A62DAA81BB810D931D932D933D936B
:1039A000A881B9810E94E42BAA81BB810D911D9150
:1039B0002D913C9140E051E060E070E00E94222DAA
:1039C000AA81BB810D931D932D933D93AA81BB8149
:1039D0000D911D912D913C91A881B981AD90BC9024
:1039E000A9EDB0E0AA0DBB1D4C915527662777279E
:1039F0000E94A62DAA81BB810D931D932D933D930B
:103A0000AA81BB810D911D912D913C91AE81BF8109
:103A10000D931D932D933C9386E0481A8827580AEE
:103A20002496089580E0A881B9818C930027BB2754
:103A3000A0E38C9183FB0EF401E040E0041711F049
:103A40000C94261D82E0A881B9818C930027BB27A6
:103A5000A0E38C9184FB0EF401E040E0041711F028
:103A60000C94361D81E0A881B9818C930027BB2777
:103A7000A3E38C9181FB0EF401E040E0041711F008
:103A80000C94461D83E0A881B9818C930027BB2745
:103A9000A3E38C9181FB0EF401E040E0041781E088
:103AA00009F080E08F930027BB27A0E38C9183FB74
:103AB0000EF401E040E0041781E009F080E09F91FE
:103AC0008923882311F40C94691D84E0A881B981AD
:103AD0008C93089581E00E94122D81E00E94122DA6
:103AE00082E00E94122D0027AFECB0E08C9183FBA6
:103AF0000EF401E041E0041711F00C94951D80E0F4
:103B0000AC81BD818C930027BB27A9E38C9185FBF9
:103B10000EF401E040E0041711F00C94931D81E0D5
:103B2000AC81BD818C930C94951E5398549880E081
:103B300081BB909A919AEF93FF93E0EFF1E00E949E
:103B4000D72CFF91EF9180E0AC81BD818C93002751
:103B5000BB27A0E38C9180FB0EF401E040E004174A
:103B600011F00C94B71D81E0AC81BD818C930027CE
:103B7000BB27A0E38C9181FB0EF401E040E0041729
:103B800011F00C94C81DAC81BD818C918E5F8C931B
:103B90000027BB27A9E38C9185FB0EF401E040E0F0
:103BA000041711F00C94D91DAC81BD818C918C5FF0
:103BB0008C930027BB27A9E38C9184FB0EF401E0D2
:103BC00040E0041711F00C94EA1DAC81BD818C918A
:103BD000885F8C93AC81BD810C91003018F011F09E
:103BE0000C94F41D0C944D1E85E090E00E94032D72
:103BF00080E0AA81BB818C930027BB27A0E38C9136
:103C000080FB0EF401E040E0041711F00C940C1E50
:103C100081E0AA81BB818C930027BB27A0E38C9114
:103C200081FB0EF401E040E0041711F00C941D1E1E
:103C3000AA81BB818C918E5F8C930027BB27A9E35F
:103C40008C9185FB0EF401E040E0041711F00C9418
:103C50002E1EAA81BB818C918C5F8C930027BB2781
:103C6000A9E38C9184FB0EF401E040E0041711F00D
:103C70000C943F1EAA81BB818C91885F8C93AA8192
:103C8000BB814C91AC81BD810C91041711F40C9453
:103C90004D1E80E0AC81BD818C93AC81BD810C91C7
:103CA000033011F00C945A1E82E0AC81BD818C93DC
:103CB0000C94901EAC81BD810C91043081E008F41D
:103CC00080E08F93AC81BD810C91073081E010F0D2
:103CD00009F080E09F918923882311F40C94761ECB
:103CE00083E0AC81BD818C930C94901EAC81BD812E
:103CF0000C91083081E008F480E08F93AC81BD81A5
:103D00000C910F3081E010F009F080E09F91892341
:103D1000882311F40C94901E84E0AC81BD818C93B7
:103D200081E081BB9198539A549AAC81BD818C916A
:103D3000AE81BF818C9384E0481A8827580A269662
:103D4000089581E00E94122D81E00E94122DAC8125
:103D5000BD818C91A881B9818C930E94CC0D88EC97
:103D600090E00E94032D5A924A9281E0A42DB52D35
:103D70008C9381E00E94CA2B0E943A29229681E00E
:103D80000E94C62BA895E9E6F0E0FA93EA930E9418
:103D9000121D22968AE090E00E94032D0091690096
:103DA000003011F00C94C21E86E990E00E94032DB1
:103DB0005A924A9280E0A42DB52D8C9381E00E9406
:103DC000CA2B0E943A29229681E00E94C62B84E6E3
:103DD00090E00E94032D5A924A9280E0A42DB52DC6
:103DE0008C9381E00E94CA2B0E943A29229681E09E
:103DF0000E94C62BA895E9E6F0E0FA93EA930E94A8
:103E0000121D22960E94CE0D5A924A9281E0A42D54
:103E1000B52D8C9381E00E94CA2B0E943A292296EC
:103E200081E00E94C62B84E690E00E94032D5A9206
:103E30004A9280E0A42DB52D8C9381E00E94CA2B7C
:103E40000E943A29229681E00E94C62B8AE090E0E7
:103E50000E94032D5A924A9280E0A42DB52D8C9396
:103E600081E00E94CA2B0E943A29229681E00E949A
:103E7000C62B0E94CC0D86E990E00E94032D009194
:103E80006900003018F011F00C94481F0C94FA1ED1
:103E900088E790E00E94032D5A924A9281E0A42D77
:103EA000B52D8C9381E00E94CA2B0E946920229636
:103EB00081E00E94C62BA881B9810C91023011F0DB
:103EC0000C94A21F00916900013011F00C946D1F39
:103ED00081E08093C1000C949B1F023011F00C9480
:103EE000851F80E08093C1005A924A9281E0A42D00
:103EF000B52D8C9381E00E94CA2B0E9469202296E6
:103F000081E00E94C62B0C949B1F033011F00C948F
:103F10009B1F83E08093C1005A924A9282E0A42DB5
:103F2000B52D8C9381E00E94CA2B0E9469202296B5
:103F300081E00E94C62BEEE0F0E0A1ECB0E07BE770
:103F40000E94392EA881B9810C91033011F00C9494
:103F5000D51F00916900013011F00C94B61FA2EC3E
:103F6000B0E08C9181608C930C94CE1F023011F0E4
:103F70000C94CE1FA2ECB0E08C918E7F8C935A9261
:103F80004A9281E0A42DB52D8C9381E00E94CA2B2A
:103F90000E946920229681E00E94C62BEFE0F0E0AB
:103FA000A2ECB0E07BE70E94392EA881B9810C9188
:103FB000013011F00C94272000916900013011F0BC
:103FC0000C94EE1FA2ECB0E08C9182608C93A2EC7A
:103FD000B0E08C918B7F8C930C942020023011F0F8
:103FE0000C940820A2ECB0E08C91897F8C935A92BB
:103FF0004A9281E0A42DB52D8C9381E00E94CA2BBA
:104000000E946920229681E00E94C62B0C942020F9
:10401000033011F00C942020A2ECB0E08C9186606B
:104020008C935A924A9282E0A42DB52D8C9381E014
:104030000E94CA2B0E946920229681E00E94C62B12
:10404000EFE0F0E0A2ECB0E07BE70E94392E0E94A6
:10405000D00DA895E9E6F0E0FA93EA930E94121DCC
:10406000229685E090E00E94032D009169000030C7
:1040700011F00C94292086E990E00E94032D5A92B9
:104080004A9280E0A42DB52D8C9381E00E94CA2B2A
:104090000E943A29229681E00E94C62B86E990E090
:1040A0000E94032D5A924A9280E0A42DB52D8C9344
:1040B00081E00E94CA2B0E943A29229681E00E9448
:1040C000C62B0E94CE0D82E0481A8827580A2496F3
:1040D000089581E00E94122D81E0A881B9818C931E
:1040E000AA81BB814C91A881B9810C91041718F069
:1040F00011F00C9496205A924A9282E0A42DB52D8C
:104100008C9381E00E94CA2B0E943A29229681E07A
:104110000E94C62B8DE790E00E94032DA881B981F3
:104120008C918F5F8C9310F40C94702081E0481A6E
:104130008827580A2296089581E00E94122D81E076
:10414000A881B9818C93A881B9810C91063018F0AF
:1041500011F00C94BF200E94CC0D8FE090E00E94E3
:10416000032D0E94CE0D84E690E00E94032DA881CD
:10417000B9818C918F5F8C9310F40C94A32081E013
:10418000481A8827580A229608950E94EF2CC39A4D
:1041900088EC90E00E94032D81B5886081BD0E946B
:1041A000FC275A924A9281E0A42DB52D8C9381E090
:1041B0000E94CA2B0E944828229681E00E94C62BAA
:1041C00081B5886181BD877F81BD84E690E00E94D2
:1041D000032DFF27E0E1FA93EA935A924A928BE08B
:1041E000A42DB52D8C9381E00E94CA2B0E94D02A69
:1041F000249681E00E94C62B013051E0150711F092
:104200000C941B215A924A92ACEBB0E08D919C9198
:10421000A42DB52D8D939C9382E00E94CA2B0E9401
:10422000E028229682E00E94C62BECE6FDE50E9483
:10423000672C0E94732C5A924A9282E3A42DB52DCA
:104240008C9381E00E94CA2B0E944828229681E02C
:104250000E94C62BC29AD89A82E390E00E94032D56
:10426000089581E00E94122D81E00E94122D8FEFAF
:10427000AA81BB818C9380E0A881B9818C93A881AD
:10428000B9810C91073018F011F00C94542191E091
:10429000AA81BB810E94E52CA881B9818C918F5F96
:1042A0008C9310F40C943F2182E0481A8827580A16
:1042B0002496089581E00E94122D81E00E94122D23
:1042C00081E00E94122D82E00E94122D82E00E9465
:1042D000122D8FEFAA85BB858C9381E0A885B985C7
:1042E0008C93A885B9850C91003418F011F00C94CA
:1042F00083210E943121A885B9858C918F5F8C9391
:1043000010F40C947121C49881E0A885B9858C9330
:10431000A885B9850C91003418F011F00C949A21FD
:104320000E943121A885B9858C918F5F8C9310F400
:104330000C9488218AE090E00E94032DA895EE81DC
:10434000FF81FA93EA935A924A9280E4A42DB52D04
:104350008C9381E00E94CA2B5A924A9200E010E0AE
:1043600020E030E0A42DB52D0D931D932D933C93AB
:1043700084E00E94CA2B0E946B27269685E00E944B
:10438000C62BAE81BF810C91013011F40C94D12168
:10439000C49AE0E7FDE50E94672C0E94732C0C9400
:1043A000882481E0AA85BB858C93A89580E090E065
:1043B000A881B9818D939C93EE81FF81FA93EA9352
:1043C0005A924A9281E4A42DB52D8C9381E00E94EB
:1043D000CA2B5A924A9200E010E020E030E0A42D6F
:1043E000B52D0D931D932D933C9384E00E94CA2B11
:1043F0000E946B27269685E00E94C62BA881B98172
:104400000E94DD2BAE81BF810C91003081E009F06C
:1044100080E08F93A881B9810D911C91003050E00C
:10442000150781E009F080E09F91892B882311F422
:104430000C94DC21C49AA881B9810D911C910030A3
:1044400050E0150711F00C942D22E8E7FDE50E94DD
:10445000672C0E94732C0C948824A89584E690E025
:104460000E94032DA895C49881E090E00E94032D3E
:10447000EE81FF81FA93EA935A924A9280E5A42D45
:10448000B52D8C9381E00E94CA2B5A924A9201E08A
:1044900010E020E030E0A42DB52D0D931D932D9359
:1044A0003C9384E00E94CA2B0E946B27269685E0ED
:1044B0000E94C62B85E090E00E94032DC49A8AE0FA
:1044C00090E00E94032DA89500E010E020E030E08D
:1044D000AAE7B0E00D931D932D933C9300E010E00C
:1044E00020E030E0A1EDB0E00D931D932D933C93BF
:1044F0000E948E2400E010E020E030E0A1EDB0E06A
:104500000D931D932D933C930027AFECB0E08C915D
:1045100086FB0EF401E041E0041711F00C949222A6
:104520000C948824A8950091E600023011F40C94B4
:10453000262380919C0280937E00A3EAB2E00D9135
:10454000112740E051E00E94182DAA81BB810D93F4
:104550001C93AA81BB810D911C91A2EAB2E04D91FE
:104560005527040F151FAA81BB810D931C93AA81A7
:10457000BB810D911C912227332740E050E061E080
:1045800070E00E94222DAAE7B0E00D931D932D93B9
:104590003D93A1EAB2E00D91112740E051E00E9465
:1045A000182DAA81BB810D931C93AA81BB810D910B
:1045B0001C91A0EAB2E04D915527040F151FAA8166
:1045C000BB810D931C93AAE7B0E00D911D912D9135
:1045D0003C91AA81BB814D915C91662777270E940F
:1045E000A62DAAE7B0E00D931D932D933D93009166
:1045F0007E000C3011F00C9400238BE080937E0041
:1046000000917E000E3011F00C9409238BE0809312
:104610007E0000917E000F3011F00C9412238BE08D
:1046200080937E00AAE7B0E00D911D912D913C9101
:10463000A1EDB0E00D931D932D933C930E948E2429
:10464000A1EDB0E00E94EB2B0C947A2300911001B5
:10465000063411F00C94502384E080937E0087E3AD
:10466000A885B9858C93A885B9850C910C3318F071
:1046700011F00C944E23A885B985AD90BB24A9ED0B
:10468000B0E0AA0DBB1D8C910E94762CA885B9853F
:104690008C918F5F8C9310F40C9433230E94732CB5
:1046A00000912C01063411F00C947A238BE0809356
:1046B0007E0083E5A885B9858C93A885B9850C9182
:1046C000073518F011F00C947823A885B985AD90C2
:1046D000BB24A9EDB0E0AA0DBB1D8C910E94762CE5
:1046E000A885B9858C918F5F8C9310F40C945D2311
:1046F0000E94732CE2E8FDE50E94672CA8E6B7E073
:10470000EEE7F0E00E94D22D0E945F2C0E94732CF5
:10471000E4E9FDE50E94672CA8E6B7E0EAE7F0E0EF
:104720000E94C62D0E945F2C0E94732C84E0A885F5
:10473000B9858C93A885B9850C910B3018F011F0D0
:104740000C94B523A885B985AD90BB24A9EDB0E044
:10475000AA0DBB1D8C910E94762CA885B9858C91E1
:104760008F5F8C9310F40C949A230E94732C809189
:10477000E70080936F00E6EAFDE50E94672CA8E65B
:10478000B7E0EFE6F0E00E94D22D0E945F2C0E947D
:10479000732C00916F00003011F00C94D1230C9415
:1047A000882400916F00003418F011F00C94DA2383
:1047B0000C94DC230C9488248091E800AE81BF81A6
:1047C0008C938091E900AC81BD818C93AC81BD81DB
:1047D0009C91AE81BF818C91ADE6B0E08D939C93AE
:1047E0008091F000AE81BF818C938091F100AC810B
:1047F000BD818C93AC81BD819C91AE81BF818C9138
:10480000A0E7B0E08D939C93A0E7B0E00D911C91E0
:10481000003050E0150711F00C9424248091FE0024
:10482000AE81BF818C938091FF00AC81BD818C9360
:10483000AC81BD819C91AE81BF818C91A0E7B0E03D
:104840008D939C930C942424A0E7B0E00D911C91CF
:10485000003050E0150711F00C9430240C9488249B
:1048600002E010E020E030E0A0E7B0E04D915C9184
:10487000662777270E94222DA2E7B0E00D931D93B3
:104880002D933D93A2E7B0E00D911D912D913C91A8
:10489000ADE6B0E04D915C91662777270E94A62D8A
:1048A000A2E7B0E00D931D932D933D93A2E7B0E0F6
:1048B0000D911D912D913C91A1EDB0E04D915D9137
:1048C0006D917C910E94A62DA2E7B0E00D931D93FF
:1048D0002D933D93E6EBFDE50E94672CA8E6B7E03B
:1048E000E2E7F0E00E94C62D0E945F2C0E94732C2C
:1048F000A2E7B0E00D911D912D913C91A1EDB0E0AA
:104900000D931D932D933C9380E0AA85BB858C93DA
:1049100087E0481A8827580A2A96089581E00E945D
:10492000122D81E00E94122D82E00E94122D82E061
:104930000E94122D8FEFAE81BF818C9391E0AE81EA
:10494000BF810E94E52C91E0AE81BF810E94E52CE1
:1049500091E0AE81BF810E94E52C91E0AE81BF81E4
:104960000E94E52C91E0AE81BF810E94E52C91E090
:10497000AE81BF810E94E52C91E0AE81BF810E9493
:10498000E52C91E0AE81BF810E94E52C91E0AE81E3
:10499000BF810E94E52C91E0AE81BF810E94E52C91
:1049A00091E0AE81BF810E94E52C91E0AE81BF8194
:1049B0000E94E52C91E0AE81BF810E94E52C91E040
:1049C000AE81BF810E94E52C91E0AE81BF810E9443
:1049D000E52C91E0AE81BF810E94E52CC49880E077
:1049E00090E0A881B9818D939C938FEF0E94F62C63
:1049F0000E94F82C0E94F72CAE81BF818C93A88175
:104A0000B9810E94DD2BAE81BF810C91003081E025
:104A100009F480E08F93A881B9810D911C91003039
:104A200050E0150781E009F080E09F91892B8823F1
:104A300011F40C94F524A881B9810D911C910030DA
:104A400050E0150711F00C943225EEEBFDE50E94C5
:104A5000672C0E94732C8091CF0080648093CF00DC
:104A60000C947F26EE81FF81FA93EA935A924A9240
:104A700081E5A42DB52D8C9381E00E94CA2B5A921A
:104A80004A92A1EDB0E00D911D912D913C91A42D84
:104A9000B52D0D931D932D933C9384E00E94CA2B5A
:104AA0000E946B27269685E00E94C62B0027AFEC5C
:104AB000B0E08C9186FB0EF401E041E0041711F0A8
:104AC0000C947225ECECFDE50E94672CA8E6B7E09B
:104AD000E1EDF0E00E94C62D0E945F2C0E94732C35
:104AE0000C947F26A895AE81BF810C91003011F007
:104AF0000C94BD2580E090E0A881B9818D939C93B2
:104B00008FEF0E94F62C0E94F82C0E94F72CAE81A9
:104B1000BF818C93A881B9810E94DD2BAE81BF81BA
:104B20000C91003081E009F480E08F93A881B98175
:104B30000D911C91003050E0150781E009F080E0F4
:104B40009F91892B882311F40C948025A881B98129
:104B50000D911C91003050E0150711F00C94BD250B
:104B6000E6EEFDE50E94672C0E94732C8091CF0039
:104B700080648093CF000C947F26AE81BF810C911E
:104B80000F3F11F00C94072680E090E0A881B981D6
:104B90008D939C938FEF0E94F62C0E94F82C0E941C
:104BA000F72CAE81BF818C93A881B9810E94DD2B47
:104BB000AE81BF810C910F3F81E009F480E08F93BB
:104BC000A881B9810D911C91003050E0150781E05A
:104BD00009F080E09F91892B882311F40C94CA2559
:104BE000A881B9810D911C91003050E0150711F09A
:104BF0000C940726E4EFFDE50E94672C0E94732CBD
:104C00008091CF0080648093CF000C947F26AE818A
:104C1000BF810C910E3F11F40C942426E2E0FEE5D6
:104C20000E94672CA8E6B7E0EE81FF810E94D22D9A
:104C30000E945F2C0E94732CC49A8091CF008064E4
:104C40008093CF000C947F2680E090E0AA81BB8106
:104C50008D939C9380E0AE81BF818C93AE81BF81A8
:104C60000C910F3F18F011F00C946626AA81BB81BD
:104C70000E94DD2B8FEF0E94F62C0E94F82C0E94E0
:104C8000F72CAA81BB81AD90BC90A9EDB0E0AA0D34
:104C9000BB1D8C93AA81BB810E94DD2B8FEF0E94EC
:104CA000F62C0E94F82C0E94F72CAA81BB81AD90B3
:104CB000BC90A9EDB0E0AA0DBB1D8C93AE81BF8165
:104CC0008C918F5F8C9310F40C942E268FEF0E94A2
:104CD000F62C0E94F82C0E94F72CAE81BF818C9399
:104CE0008FEF0E94F62C0E94F82C0E94F72CAE81C8
:104CF000BF818C93C49AA1EDB0E00E94CE2B86E0D8
:104D0000481A8827580A2896089582E00E94122D92
:104D100081E00E94122D80E0AE81BF818C930E94C1
:104D20003121C49880E090E0AA81BB818D939C934F
:104D30008FEF0E94F62C0E94F82C0E94F72CA8817D
:104D4000B9818C93AA81BB810E94DD2BA881B98196
:104D50000C91003081E009F480E08F93AA81BB813F
:104D60000D911C91003050E0150781E009F080E0C2
:104D70009F91892B882311F40C949826AA81BB81DA
:104D80000D911C91003050E0150711F00C94D526C0
:104D9000EEEBFDE50E94672C0E94732C8091CF0002
:104DA00080648093CF000C946527E881F981FA93A1
:104DB000EA935A924A9281E5A42DB52D8C9381E015
:104DC0000E94CA2B5A924A92AA85BB850D911D91C9
:104DD0002D913C91A42DB52D0D931D932D933C93B6
:104DE00084E00E94CA2B0E946B27269685E00E94D1
:104DF000C62BA881B9810C91003011F00C942C279E
:104E000080E090E0AA81BB818D939C938FEF0E94FC
:104E1000F62C0E94F82C0E94F72CA881B9818C9363
:104E2000AA81BB810E94DD2BA881B9810C91003041
:104E300081E009F480E08F93AA81BB810D911C91E0
:104E4000003050E0150781E009F080E09F91892B48
:104E5000882311F40C940627A881B9810C910F3F87
:104E600011F00C945F2780E090E0AA81BB818D93C4
:104E70009C938FEF0E94F62C0E94F82C0E94F72C36
:104E8000A881B9818C93AA81BB810E94DD2BA88166
:104E9000B9810C910F3F81E009F480E08F93AA81E2
:104EA000BB810D911C91003050E0150781E009F0A5
:104EB00080E09F91892B882311F40C943927A881D5
:104EC000B9818C91AE81BF818C9383E0481A882789
:104ED000580A2496089584E00E94122D81E00E94D1
:104EE000122D82E00E94122D8FEFAA81BB818C933C
:104EF00091E0AA81BB810E94E52C91E0A885B9854B
:104F00000E94E52CAE81BF810D911D912D913C91A8
:104F100040E052E060E070E00E94222DAC81BD8153
:104F20000D931D932D933D93AC81BD818F9314966A
:104F30008E910E94F1278E910E94F1278E910E94FE
:104F4000F1278E910E94F12785E90E94F1278F9128
:104F500080E090E0A881B9818D939C938FEF0E94AF
:104F6000F62C0E94F82C0E94F72CAA81BB818C930E
:104F7000A881B9810E94DD2BAA81BB810C910F3FD2
:104F800081E009F480E08F93A881B9810D911C9193
:104F9000003050E0150781E009F080E09F91892BF7
:104FA000882311F40C94AE27A881B9810D911C912E
:104FB000003050E0150711F00C94E927E0E1FEE520
:104FC0000E94672C0E94732C8091CF008064809394
:104FD000CF00AA81BB818C91AA85BB858C930C9450
:104FE000F6278FB9779BFECF8FB1089587E0481AD7
:104FF0008827580A269608955A924A9284E298E0A1
:10500000A42DB52D8D939C9382E00E94CA2B5A92B9
:105010004A9280E0A42DB52D8C9381E00E94CA2B8A
:105020000E94752A249683E00E94C62BEF93FF937B
:10503000ECE8F1E00E94D72CFF91EF91BB27A0E3B1
:105040008C9182FBDEF789E190E00E94032D5A9259
:105050004A9280E298E0A42DB52D8D939C9382E036
:105060000E94CA2B5A924A9280E0A42DB52D8C93AF
:1050700081E00E94CA2B0E94752A249683E00E9438
:10508000C62B89E190E00E94032D0E94FD2808951F
:1050900082E00E94122D00E011E0AA81BB814D91B7
:1050A00055270E94182DA881B9810D931C93A881C2
:1050B000B9810D911C91AA81BB814D915527040F97
:1050C000151FA881B9810D931C935A924A92AA8107
:1050D000BB818D919C91A42DB52D8D939C9382E0E5
:1050E0000E94CA2B5A924A928BE0A42DB52D8C9324
:1050F00081E00E94CA2B0E94752A249683E00E94B8
:10510000C62B5A924A9280E298E0A42DB52D8D9339
:105110009C9382E00E94CA2B5A924A9280E0A42D6E
:10512000B52D8C9381E00E94CA2B0E94752A24968B
:1051300083E00E94C62B82E0481A8827580A2296EC
:10514000089582E00E94122D00E110E0AC81BD8143
:105150004D9155270E94182DA881B9810D931C935C
:10516000A881B9810D911C91AA81BB814D915527D0
:10517000040F151FA881B9810D931C935A924A926E
:10518000AA81BB818D919C91A42DB52D8D939C936B
:1051900082E00E94CA2B5A924A9282E0A42DB52D39
:1051A0008C9381E00E94CA2B0E94752A249683E08A
:1051B0000E94C62B82E0481A8827580A2296089532
:1051C0005A924A92AA81BB818D919C91A42DB52DB2
:1051D0008D939C9382E00E94CA2B5A924A9283E05C
:1051E000A42DB52D8C9381E00E94CA2B0E94752AB4
:1051F000249683E00E94C62B089581E00E94122D20
:1052000081E00E94122DC49AD898C29880E0A881AB
:10521000B9818C9380E0AA81BB818C93AA81BB81E8
:105220000C910F3118F011F00C94322991E0A88103
:10523000B9810E94E52C91E0A881B9810E94E52CFA
:1052400091E0A881B9810E94E52C91E0A881B98103
:105250000E94E52CAA81BB818C918F5F8C9310F406
:105260000C940E29C29AD89A82E0481A8827580AC4
:105270002496089581E00E94122D5A924A9280E26B
:1052800098E0A42DB52D8D939C9382E00E94CA2BAB
:105290005A924A9280E0A42DB52D8C9381E00E9411
:1052A000CA2B0E94752A249683E00E94C62BAA81ED
:1052B000BB810C91003011F00C946D295A924A92E6
:1052C00080E0A42DB52D8C9381E00E94CA2B0E9412
:1052D000E729229681E00E94C62BAA81BB810C910E
:1052E000013011F00C9483295A924A9285E6A42D3C
:1052F000B52D8C9381E00E94CA2B0E94E72922964B
:1053000081E00E94C62BAA81BB810C91023011F072
:105310000C94B0295A924A9283E6A42DB52D8C9311
:1053200081E00E94CA2B0E94E729229681E00E9418
:10533000C62B88EC90E00E94032D5A924A9280E09E
:10534000A42DB52D8C9381E00E94CA2B0E94E729E1
:10535000229681E00E94C62B82E390E00E94032DFA
:10536000AA81BB810C91033011F00C94D9295A9277
:105370004A9282E6A42DB52D8C9381E00E94CA2B1F
:105380000E94E729229681E00E94C62B80E991E0E5
:105390000E94032D5A924A9280E0A42DB52D8C9341
:1053A00081E00E94CA2B0E94E729229681E00E9498
:1053B000C62B8AE090E00E94032D8AE090E00E94D4
:1053C000032D81E0481A8827580A2296089581E023
:1053D0000E94122DC49AD898C298AA81BB810C91C0
:1053E000003018F011F00C94F7290C94312A83E561
:1053F000A881B9818C9391E0A881B9810E94E52CA4
:105400008FEEA881B9818C9391E0A881B9810E9427
:10541000E52C8EE6A881B9818C9391E0A881B981B1
:105420000E94E52C91E0AA81BB810E94E52C80E0DE
:10543000A881B9818C9391E0A881B9810E94E52C63
:1054400091E0A881B9810E94E52C91E0A881B98101
:105450000E94E52C91E0A881B9810E94E52C0C9472
:105460006D2A85E4A881B9818C9391E0A881B981E6
:105470000E94E52C88E7A881B9818C9391E0A881EE
:10548000B9810E94E52C89E6A881B9818C9391E0CD
:10549000A881B9810E94E52C84E7A881B9818C9309
:1054A00091E0A881B9810E94E52C80E0A881B981B2
:1054B0008C9391E0A881B9810E94E52C91E0A881AC
:1054C000B9810E94E52C91E0A881B9810E94E52C68
:1054D00091E0A881B9810E94E52CC29AD89A81E016
:1054E000481A8827580A2296089581E00E94122DB2
:1054F000C29AD8985A924A9282E0A42DB52D8C93E4
:1055000081E00E94CA2B0E942A2B229681E00E94F1
:10551000C62B5A924A92AC81BD818C91A42DB52D97
:105520008C9381E00E94CA2B0E942A2B229681E054
:105530000E94C62BAC81BD8111968C91A881B98146
:105540008C935A924A92AA81BB818C91A42DB52D3D
:105550008C9381E00E94CA2B0E942A2B229681E024
:105560000E94C62BAC81BD818C91A881B9818C939E
:105570005A924A92AA81BB818C91A42DB52D8C930D
:1055800081E00E94CA2B0E942A2B229681E00E9471
:10559000C62BD89A81E0481A8827580A229608957F
:1055A00081E00E94122D81E00E94122D82E00E9473
:1055B000122DC29AD8985A924A9283E0A42DB52D02
:1055C0008C9381E00E94CA2B0E942A2B229681E0B4
:1055D0000E94C62B5A924A92A885B9858C91A42D17
:1055E000B52D8C9381E00E94CA2B0E942A2B229613
:1055F00081E00E94C62BEC81FD81FA93EA930E9420
:10560000302B2296EA81FB81FA93EA930E94302B99
:105610002296D89AAC81BD810D91112740E051E0CE
:105620000E94182DA881B9810D931C93A881B9817E
:105630000D911C91AA81BB814D915527040F151F17
:10564000A885B9850D931C9384E0481A8827580AC9
:105650002696089591E0A881B9810E94E52C0895CD
:1056600081E00E94122D91E0A881B9810E94DA2C7C
:10567000A881B9818C91AA81BB818C9381E0481A61
:105680008827580A2296089582E00E94122D81E010
:105690000E94122DC49ABB27A0E38C9182FBDEF7F7
:1056A000C298AC81BD810D911C91003052E015076C
:1056B00011F00C94932B81E090E0AA81BB818D9333
:1056C0009C9380E0A881B9818C93A881B9810C91C9
:1056D0000F3018F011F00C94912BBB27A0E38C91A4
:1056E00082FBDEF790E2AA81BB81AD90BC90A9ED70
:1056F000B0E0AA0DBB1D0E94E52CAA81BB810D91D3
:105700001C9140E250E0040F151FAA81BB810D934C
:105710001C93A881B9818C918F5F8C9310F40C94A9
:10572000652B0C94BF2B81E090E0AA81BB818D9307
:105730009C93AC81BD814D915C91AA81BB810D91FF
:105740001C910417150718F011F00C94BF2BBB2700
:10575000A0E38C9182FBDEF7C29A91E0AA81BB8123
:10576000AD90BC90A9EDB0E0AA0DBB1D0E94E52C48
:10577000AA81BB810E94DD2B10F40C94992BC29A54
:1057800083E0481A8827580A24960895481A8827DB
:10579000580A0895480E8827581E08950D911D91A6
:1057A0002D913C9181E0080F8827181F281F381F72
:1057B0003C932E931E930E930895ED91FC91EF5F11
:1057C000FF4FFC93EE930895ED91FC91E150F04072
:1057D000FC93EE9308950D911D912D913C910150F4
:1057E0001040204030403C932E931E930E9308951A
:1057F0004091DB025091DC020DE815E30E940C2C75
:1058000049E156E3040F151F0093DB021093DC02FD
:10581000498158810C94322C09D00E94182D00FC2B
:1058200010D0089503D01ED001F8F9CF0024E894D9
:1058300057FF02C009D0689400F80BD010F801247B
:10584000089502D009D00895509540954F5F5F4F5D
:105850000895E89417FF0895009510950F5F1F4F66
:1058600068940895352F242FE894452B11F46894FB
:105870000895512F402F0027112780E1440F551F15
:10588000001F111F021B130B416018F4020F131F9E
:105890004E7F8A9599F708958F938D918823E9F724
:1058A00011978F91089581E05F9B8827089588273D
:1058B0005F9B089500C05F9BFECF8CB10895A8E662
:1058C000B7E08D91882311F011D0FBCF08950E948D
:1058D000542D802D11F00AD0FACF08958D9106D065
:1058E0003A95E1F708958DE001D08AE05D9BFECF07
:1058F0008CB9089588EE93E086D03197D9F7089552
:1059000000FC05D0089530D005D001F8F9CF37D08C
:105910003FD00895842F952FA62FB72FE894452BBD
:10592000462B472B11F468940895402F512F622F76
:10593000732F0027112722273327F0E2440F551F2A
:10594000661F771F001F111F221F331F081B190B13
:105950002A0B3B0B416028F4080F191F2A1F3B1F1D
:105960004E7FFA9559F708950024E89477FF02C016
:1059700006D0689400F809D010F80124089512D0D8
:105980004F5F5F4F6F4F7F4F0895E89437FF089543
:1059900000951095209530950F5F1F4F2F4F3F4F6B
:1059A0006894089540955095609570950895319745
:1059B000F1F708950E94F62C8C910E94F82C8D939B
:1059C0009A95D1F70E94F72C08950E94F62C8D919C
:1059D0000E94F82C9A95D9F70E94F72C0895BF9A47
:1059E000BE98C69ABD9A80E58DB908950895089528
:1059F0008FB9779BFECF8FB10895689462F80895B0
:105A0000E89462F80895EF93FF93EE27E82BE92BD3
:105A100031F0E0EDF7E03197F1F70197D1F7FF9121
:105A2000EF9108955A924A92480E8827581E089579
:105A30000F92B801469F8001479F100D569F100D91
:105A40000F9008950F921F922F92C801D901489F7D
:105A500080014A9F90014B9F202C499F100D211DD2
:105A6000321D5A9F202C589F100D211D321D599F09
:105A7000200D311D689F200D311D699F300D789FCD
:105A8000300D2F901F900F9008950E94542D0D926D
:105A90000020D9F70895369A3699FECF369A36996E
:105AA000FECF84B195B10895C89531960020089530
:105AB000819104D08D938823D9F70895813618F009
:105AC0008B3708F48F7D089580E30EF48395089555
:105AD0002E2E3F2E992781918D3209F093958823A0
:105AE000D1F79A95E22DF32D112361F0091718F0E3
:105AF00011F0101B01C0191B28F021F080E28D93DA
:105B00001A95E9F780818D3219F48D93319604C08E
:105B1000222311F08BE28D93091738F031F0091B25
:105B200021F080E38D930A95E9F781918D93882385
:105B3000E1F7332351F0EA2FFB2F319633958E9105
:105B400082933A95E1F78EE28C930895040F151F26
:105B5000261F371F0895041B150B260B370B0895BE
:105B600004171507260737070895000F111F221F76
:105B7000331F089500951095209530950F5F1F4FA6
:105B80002F4F3F4F0895019110810EC00191119147
:105B9000219130810BC00191108117FF05C03FEFAB
:105BA0002FEF04C0008111272227332737FF03C0BE
:105BB000E1DF8DE28D93CF93DF93CF92DF92EF926F
:105BC000AA24BB24CC24DD24EE2440E2CAE0DD2755
:105BD00055E093E38881890F87FD9F7083FD907F57
:105BE000891B89935A95A9F7C0DFAA1CBB1CCC1C42
:105BF000DD1CEE1C4A9551F7E894EFE0FF278291F7
:105C00000ED0EB30E0F71EF068948A2D0CD0882778
:105C10008D93EF90DF90CF90DF91CF910895982FE3
:105C2000829501D0892F8F70805D26F0803309F432
:105C3000089568948D93089588278D930895819190
:105C40008D938823E1F7089509919191992351F05B
:105C50008A95D9F7319781918D930A9519F0882308
:105C6000D1F70895E9CFE199FECFEEBBFFBB3196A6
:105C7000089591E001C092E07B3751F47FB7F8942A
:105C8000F2DF8D918DBBE29AE19A9A95C9F77FBFB9
:105C90007727089591E001C092E0E5DFE09A8DB3A7
:105CA0008D939A95D1F70895FF93881BF9E0001F13
:105CB000FA9511F4FF910895881F841B18F4840F3E
:105CC0008894F5CF0894F3CF689401C0E894AF931B
:105CD000BF938D9116F0919103C00E94542D902D89
:105CE000891718F011F48823A1F7BF91AF91089597
:105CF0004D50335354414D50205265616C69747955
:105D00002D53797320342E356E6F707269005300F5
:105D10005000454570726F6D20002C004D4D4320A2
:105D2000696E697420007265747279202E2E2E00BF
:105D300044535020696E697420004F005A00590086
:105D400057005200480021004E0042005800440015
:105D5000450056004D00540049004C00434F4E464C
:105D6000494700002000442000002E006F6B000017
:105D70004E6F2063617264004261642063617264EB
:105D80000000506172746974696F6E207479706577
:105D9000203A0000506172746974696F6E207374E8
:105DA0006172743A0000536563742F636C75737489
:105DB000657220203A00526F6F74203A00005265DD
:105DC0006164206572726F722031000052656164F7
:105DD000206572726F722032206F6E20736563745B
:105DE0006F723A20000052656164206572726F72B2
:105DF0002033000052656164206572726F72203436
:105E0000000052656164206572726F722035000077
:0E5E1000526561642074696D656F75740000E1
:00000001FF
